:0A0B3C000001020203030404050592
:100546005010C0C0F9A4B0999282F880988883C6EA
:03055600A1868EED
:1002B700E4F513F512F511F510C203C200C202C22C
:1002C700011206377E077F008E238F24752B077553
:1002D7002C1275210775221C752907752A4A752D59
:1002E70007752E78EE54C070030203B875140075B5
:1002F70015808E168F17C374C09FFF74079ECF2477
:1003070002CF3400FEE48F0F8E0EF50DF50CF50BC2
:10031700F50AF509F508AF0FAE0EAD0DAC0CAB0B3A
:10032700AA0AA909A808C3120B205033E517250B01
:10033700F582E516350AF583E0FFE515250BF5820D
:10034700E514350AF583EFF0E50B2401F50BE435E9
:100357000AF50AE43509F509E43508F50880B78593
:10036700142385152474002480FF740734FFFEC30B
:10037700E52C9FF52CE52B9EF52BC3E5269FF5264F
:10038700E5259EF525C3E5289FF528E5279EF52752
:10039700C3E5229FF522E5219EF521C3E52A9FF5B6
:1003A7002AE5299EF529C3E52E9FF52EE52D9EF515
:1003B7002DD2E843D82090E668E0440BF090E65C45
:1003C700E0443DF0000000000000E4F5A20000005A
:1003D700D2AF90E680E020E105D2041206D090E685
:1003E70080E054F7F0538EF8C20390E6C2E054FB66
:1003F700F000000000000090E6187410F000000004
:1004070090E61A7408F000000090E6017403F0000B
:100417000000300105120080C2013003F5120B5AAB
:1004270050F0C203120A7B20001690E682E030E704
:1004370004E020E1EF90E682E030E604E020E0E42B
:080447001209FC120B5C80CAD3
:0B0B310090E50DE030E402C322D32267
:1000800090E6B9E0700302013F1470030201BC2442
:10009000FE700302023F24FB700302013914700357
:1000A00002013314700302012714700302012D248E
:1000B0000560030202A3120B5E40030202AF90E64A
:1000C000BBE024FE602714603824FD601114602713
:1000D00024067050E52390E6B3F0E524803C120B33
:1000E00031503EE52B90E6B3F0E52C802DE52590D0
:1000F000E6B3F0E5268023E52790E6B3F0E5288017
:100100001990E6BAE0FF120A28AA06A9077B01EABD
:10011000494B600DEE90E6B3F0EF90E6B4F00202CA
:10012000AF02029E02029E120B0E0202AF120B4E93
:100130000202AF120B460202AF120AFC0202AF1219
:100140000B6040030202AF90E6B8E0247F60151414
:10015000601924027063A200E43325E0FFA202E4E8
:10016000334F8041E490E740F0803F90E6BCE0549C
:100170007EFF7E00E0D394807C0040047D018002FD
:100180007D00EC4EFEED4F243CF582740B3EF58372
:10019000E493FF3395E0FEEF24A1FFEE34E68F8277
:1001A000F583E0540190E740F0E4A3F090E68AF094
:1001B00090E68B7402F00202AF02029E120B6240C4
:1001C000030202AF90E6B8E024FE6016240260034A
:1001D0000202AF90E6BAE0B40105C2000202AF022B
:1001E000029E90E6BAE0705590E6BCE0547EFF7E39
:1001F00000E0D394807C0040047D0180027D00EC0F
:100200004EFEED4F243CF582740B3EF583E493FFE4
:100210003395E0FEEF24A1FFEE34E68F82F583E014
:1002200054FEF090E6BCE05480131313541FFFE01B
:10023000540F2F90E683F0E04420F08072805F122C
:100240000B64506B90E6B8E024FE60192402704EF7
:1002500090E6BAE0B40104D200805490E6BAE064BB
:1002600002604C803990E6BCE0547EFF7E00E0D313
:1002700094807C0040047D0180027D00EC4EFEED08
:100280004F243CF582740B3EF583E493FF3395E0F5
:10029000FEEF24A1FFEE34E68F82F583800D90E619
:1002A000A08008120A53500790E6A0E04401F090A5
:0602B000E6A0E04480F02E
:0102B6002225
:03003300020B5667
:040B560053D8EF324F
:100700001201000200000040E4E411220000010296
:1007100000010A06000200000040010009022E004C
:1007200001010080320904000004FF0000000705F9
:10073000020200020007050402000200070586020B
:100740000002000705880200020009022E000101D4
:100750000080320904000004FF00000007050202C7
:100760004000000705040240000007058602400023
:100770000007058802400000040309041C0341002F
:100780007300740072006900620061006E006B000B
:10079000320030003000360028035800500044007A
:1007A00028004200610073006500640020006F00B3
:1007B0006E002000410058005500500050002900F4
:0207C000000037
:100559005010B0C0F9A4B0999282F880988883C6E7
:10056900A1868E4110ABFF4110AD004110AEFF4195
:0705790010AC004110AF00BF
:1006370090E600E054E74410F000000090E60474F0
:1006470080F00000007406F0000000E4F0000000F5
:1006570090E610F090E611F000000090E613F0002D
:10066700000090E615F090E61074A0F090E611F007
:1006770000000000000090E61274AAF0000000904D
:10068700E61474EAF000000090E6047480F00000BD
:10069700007404F0000000E4F000000090E64974E4
:1006A70082F0000000F000000090E6187410F000DF
:1006B700000090E61A7408F090E6917480F000004C
:0906C70000F000000043AF012225
:020B5A00D322A4
:020B5C00D322A2
:020B5E00D322A0
:080B460090E6BAE0F51BD32292
:100AFC0090E740E51BF0E490E68AF090E68B04F07A
:020B0C00D322F2
:080B4E0090E6BAE0F51AD3228B
:100B0E0090E740E51AF0E490E68AF090E68B04F068
:020B1E00D322E0
:020B6000D3229E
:020B6200D3229C
:020B6400D3229A
:100A530090E6B9E0242F600D04701990E604E0FFDE
:100A6300430780800890E604E0FF53077F000000FF
:070A7300EFF08002D322C363
:010A7A002259
:100AA000C0E0C083C082D2015391EF90E65D740133
:080AB000F0D082D083D0E032C7
:100AD000C0E0C083C0825391EF90E65D7404F0D013
:060AE00082D083D0E03259
:100AE600C0E0C083C0825391EF90E65D7402F0D0FF
:060AF60082D083D0E03243
:1009C600C0E0C083C082852925852A2685268285A2
:1009D6002583A37402F08521278522288528828510
:1009E6002783A37407F05391EF90E65D7410F0D05F
:0609F60082D083D0E03244
:100AB800C0E0C083C082D2035391EF90E65D740812
:080AC800F0D082D083D0E032AF
:1007C200C0E0C083C08290E680E030E7208521252A
:1007D200852226852682852583A37402F085292712
:1007E200852A28852882852783A37407F05391EFF1
:0D07F20090E65D7420F0D082D083D0E0321C
:0106FF0032C8
:0107FF0032C7
:010B6600325C
:010B6700325B
:010B6800325A
:010B69003259
:010B6A003258
:010B6B003257
:010B6C003256
:010B6D003255
:010B6E003254
:010B6F003253
:010B70003252
:010B71003251
:010B72003250
:010B7300324F
:010B7400324E
:010B7500324D
:010B7600324C
:010B7700324B
:010B7800324A
:010B79003249
:010B7A003248
:010B7B003247
:010B7C003246
:010B7D003245
:010B7E003244
:010B7F003243
:010B80003242
:010B81003241
:010B82003240
:010B8300323F
:010B8400323E
:010B8500323D
:10098A00C0E0C083C08290E6D1E09010ACF090E65F
:10099A00D0E4F000000090E6D17402F000000053A9
:1009AA0091BF00000090E66104F000000090E69913
:0C09BA0004F075BB06D082D083D0E03280
:010B8600323C
:03004300020800B0
:03005300020800A0
:10080000020AA000020AE600020AD000020AB800AA
:100810000209C6000207C2000206FF000207FF002D
:10082000020B6600020B6700020B6800020B6900F6
:10083000020B6A00020B6B00020B6C00020B6D00D6
:10084000020B6E000207FF00020B6F00020B70002C
:10085000020B7100020B7200020B7300020B74009A
:10086000020B75000207FF000207FF000207FF00EE
:10087000020B7600020B7700020B7800020B790066
:10088000020B7A00020B7B00020B7C00020B7D0046
:10089000020B7E00020B7F00020B8000020B810026
:1008A000020B8200020B8300020B8400020B850006
:0808B00002098A00020B860018
:1009FC0090E682E030E004E020E60B90E682E03006
:100A0C00E119E030E71590E680E04401F07F147EB8
:0C0A1C000012094490E680E054FEF02235
:1006D00030040990E680E0440AF0800790E680E06C
:1006E0004408F07FDC7E0512094490E65D74FFF05B
:0F06F00090E65FF05391EF90E680E054F7F02230
:020A2800A9071C
:100A2A00AE2DAF2E8F828E83A3E064037017AD01C3
:100A3A0019ED7001228F828E83E07C002FFDEC3E3F
:080A4A00FEAF0580DFE4FEFFB2
:010A52002281
:100A7B0090E682E044C0F090E681F04387010000ED
:040A8B000000002245
:100944008E188F1990E600E054187012E5192401EE
:10095400FFE43518C313F518EF13F519801590E665
:1009640000E05418FFBF100BE51925E0F519E51850
:1009740033F518E5191519AE18700215184E6005EF
:06098400120A8F80EE2232
:100A8F007400F58690FDA57C05A3E582458370F97A
:010A9F002234
:1005800060801000011113213C01010703030305E2
:10059000010000000C0D0C0C0E0E0E0E410000367A
:1005A0000900003F010A013B0101010701010201AD
:1005B0000000000002020000020202024049004066
:1005C0000000003F010101010101010700000000DE
:1005D000000000000E0E0E0E0E0E0E0E00000000AB
:1005E0000000003F0139010101010107000302027F
:1005F000020202020E0E0E0E0E0E0E0E002D000056
:100600000000003F60241087000000000000000090
:1006100000000000000000000000833611170004F5
:10062000030201813616170004030201471080E01F
:0606300000000ECE4E009A
:10044F0090E60174CEF090E6F574FFF0901080E026
:10045F0090E6F3F0901081E090E6C3F0901082E008
:10046F0090E6C1F0901083E090E6C2F0901085E026
:10047F0090E6C0F0901086E090E6F4F075AF077448
:10048F0010F59A7400F59B759DE4E4F59EFF90E6D8
:10049F007BE090E67CF00FBF80F490E67174FFF084
:1004AF00F5B490E672E04480F043B680000000E4BB
:1004BF0090E6C4F000000090E6C5F0901087E09041
:1004CF00E6C6F0901088E090E6C7F0901089E090B3
:1004DF00E6C8F090108AE090E6C9F090108BE0909B
:1004EF00E6CAF090108CE090E6CBF090108DE09083
:1004FF00E6CCF090108EE090E6CDF000000090E694
:10050F00D27401F000000090E6E204F00000000059
:10051F00000090E6EB14F000000000000000000067
:10052F0090E6C0F090E6C1F090E6247408F0000069
:06053F0000E490E625F047
:010545002293
:030000000208B83B
:0C08B800787FE4F6D8FD75812E0208FF61
:100B2000EB9FF5F0EA9E42F0E99D42F0E89C45F02B
:010B300022A2
:1008C4000202B7E493A3F8E493A34003F68001F291
:1008D40008DFF48029E493A3F85407240CC8C33335
:1008E400C4540F4420C8834004F456800146F6DF04
:1008F400E4800B0102040810204080900546E47E49
:10090400019360BCA3FF543F30E509541FFEE493F8
:10091400A360010ECF54C025E060A840B8E493A3BF
:10092400FAE493A3F8E493A3C8C582C8CAC583CAEA
:10093400F0A3C8C582C8CAC583CADFE9DEE780BEA2
:0106360000C3
:00000001FF
